:100000004A230D3084007C280B1D09009000030E4C
:100010008F008312851D0E2891011328110F910066
:100020004120FF309C00051E172892011C28120F4A
:1000300092004120FF309C00061C202893012328B9
:10004000130F930041201A081B0403192C289B0F3F
:100050002C289A0F2C289D151708031D9703180AA2
:10006000031935281808031D98031C0803193B2899
:100070009C0B3B281D160F0E8300900E100E0B11CB
:100080000900FB309A00B4309B000800820754340A
:1000900058340034523458340034583400344C341A
:1000A0000034203400342034443449345334503440
:1000B0004C3441345934203400344D3455344C34AC
:1000C000543400344D344134583400344D344934C0
:1000D0004E34203400342034563443344F342034EA
:1000E0004F34463446345334453454342034003489
:1000F0004D3448347A34003443308C008001840A13
:100100008C0B7E288316183085000330860004305F
:10011000810083128101A0308B00FE30860086149E
:100120000722061C9D166E2341209D11C730DF213A
:100130000830E5216B219D1994287A23051DA428F8
:100140001D1F9D171D17A7281D1B9D171D13C630AA
:10015000DF2106301D1DAF281F1FAF280A30E52103
:100160009D1FB5289C1BCD289D131D1FC228243020
:1001700035235223283043232E232A30432321239F
:100180002430CC282630352352232E3043232E23EF
:1001900030304323212326303C23BE217D219D1E68
:1001A0009B28D723191C9B28D9210C30E521163018
:1001B000E5219D199428BE21A8231918A30AB92363
:1001C0001918A303013023020318E8280130A30003
:1001D00015302302031CEE281430A300C2012308AB
:1001E000C3000A304302031CF828C300C20AF128E6
:1001F0008E30DF214208303ED5214308303ED521E4
:100200009F23191CD928DE211F30E5210330E52169
:100210000C30E5216B219D199428BE2128307221D4
:1002200028303C237D219F23191C0B29DE211B3004
:10023000E5219D199428BE212A30352352232830E8
:1002400070212A303C237D219F23191C1929DE218E
:100250000330E5212430E5219D199428BE212C305E
:10026000AD212C303C237D219F23191C2C29DE211C
:100270001F30E5210030E5210C30E5219D1994283F
:10028000BE212E3072212E303C237D219F23191C4C
:100290003E29DE211B30E5219D199428BE213030F6
:1002A000352352232E30702130303C237D219F2373
:1002B000191C4C29DE210030E5212430E5219D194F
:1002C0009428BE213230AD2132303C237D219F2342
:1002D000191C5F299428C230DF213130E521080044
:1002E0004323762935235223B901BA012E234D30F9
:1002F000B9008030BA00212308009D103709C039A9
:10030000031D89299D14B709B8090130B8070318DE
:10031000B70A2308B6000310B60DB60DB6073608A7
:10032000B6000310B60DB60DB6073608B6000310BA
:10033000B60DB60DB607EA2292228030DF21413099
:10034000840008308C000008D521840A8C0BA32976
:10035000C030DF210008D521080035238030B706E2
:1003600052238130B9009030BA0021237E30B90089
:100370007030BA002E238030B70608004122051DD8
:10038000C7292430352321303C232C30CC2926307A
:10039000352321303C23323043230A231D222130D0
:1003A00035230800D421D4212030A100A2008615D5
:1003B000EE290130DF2118304B2308008130A100E5
:1003C000A2008611EE2186150800A0004620FF3904
:1003D00003190800D5212008013EE52905118316DF
:1003E0000130860083120615F030A10506080E398B
:1003F0002104860006110615A20EF030A20506089B
:100400000E392204860006114B308E220800860128
:100410001822182218222830860006114A23283074
:10042000DF210830DF21D9210630DF210C30DF2920
:100430004A2338308600061108009E101D156723D8
:100440004A30B900B030BA002E234B30B900F0303A
:10045000BA00212334304323182303193E2A3430B1
:100460003C237322C2306522370865223808652292
:100470008E3065220030652278221F139E181D11D0
:1004800008001F1F472A1808031D592A62227322D9
:10049000C330652208308C008D2205148D22060C95
:1004A0009F0D05108C0B4C2A89227F2278221F1B5E
:1004B0006222051D1F1F602A1D1D602A861008006C
:1004C000861408006E3098000800A00008308C00E8
:1004D000A00D03188922031C84227F228C0B682A1A
:1004E00089227F220800051489228D228422812AF4
:1004F00084228D2205148D2289228D2208008D22CE
:1005000005148D22051008008510831685108312AE
:10051000080083168514831208000F308D008D0BA0
:100520008F2A0800031018308C00C201C401C601D4
:10053000C901BF0DBE0DBD0DC90DC60DC40DC20D47
:100540008C0BC52A490EC800460EC500440EC300D8
:10055000420EC1001D104130DA224230DA2243300F
:10056000DA224430DA224530DA221D144630DA220B
:10057000A530C7004830DA224930DA229D1C080035
:10058000400884002D30800008004930CE224630DB
:10059000CE224430CE224230CE22992A840003302B
:1005A0000007A000A019800030300007A000A01BA9
:1005B0008000080084000F3000050319E32A303E54
:1005C00080001D1408001D18DF2A20308000040858
:1005D000C0000800BF013708BD003808BE00083061
:1005E0008C00B60C0318F92A8C0BF12ABD01BE0150
:1005F00008000310042BB60C031C042B3808BE079C
:1006000037080318370FBD07BD0CBE0CBF0C8C0B91
:10061000FB2A08003A08B80739080318390FB7074A
:1006200008003A08B8023908031C390FB70208005D
:100630003A083802A0003908031C390A370220049E
:1006400008003908BB003A08BC000130BA0703189B
:10065000B90A1823031C08003B30322B1823031857
:100660000800393035239E14080084000008B700C4
:10067000840A0008B8000800840037088000840A53
:1006800038088000080084000008B900840A0008C7
:10069000BA00080076308D008E018E0B4D2B8D0B2D
:1006A0004D2B0800B9010130061C1430BA00B023EC
:1006B00019180A23C123191811230230061CC83047
:1006C000BA00A82319180A23B923191811233709C6
:1006D000C039031D0800B701B801080089012330A3
:1006E000840011308C008D238000890A840A8C0BD1
:1006F000732B08001D1E08001D1289012330840081
:1007000011308C008D2300020319882B00089223DE
:10071000890A840A8C0B822B080083160814831222
:10072000080808008800831608120815553089004B
:10073000AA3089008814081E9B2B831208001E30E3
:10074000A000160899001302CA2313089600080097
:1007500064301102031CB02B463091006630B12B7F
:100760003C30A000140899001102CA23110894001B
:10077000080064301202031CC12B46309200663020
:10078000C22B3C30A000150899001202CA2312089F
:10079000950008000318D42B1908053C0318D42B26
:1007A00019082002FF30031C0301990008009F2351
:1007B000191C080017080319DE2B080019309700D0
:0207C000D42B38
:02400E00FA3F77
:1042000001004F00A400510038000F00A0005D0025
:10421000C000000000000F00A0005D00C000000012
:0242200000009C
:00000001FF
